:020000040000FA
:0400000019280000BB
:020008000528C9
:06000A00F0000308F800FD
:100010000A08F9000408FA008B1C0F28000083016D
:100020007A08840079088A0078088300F00E700E40
:1000300009008312031385018601870183160313C8
:100040008501FF308700860006309F00831203136E
:100050008501F7010608F300F3080319F30A0708FE
:10006000F400F4080319F40AFF30850045207708EE
:1000700073020319051077087402031985104B20C9
:10008000F70A031D372850202A28FF30F50000000A
:10009000F50B472808000830F500F50B4D2808003F
:1000A0004630F500FF30F60000000000F60B542843
:0600B000F50B52280800C8
:0400B60000340034DE
:02400E007A3FF7
:00000001FF
